:100000000C9401040C9432040C9432040C943204C9
:100010000C9432040C9432040C9432040C94320488
:100020000C9432040C9432040C9432040C94320478
:100030000C9432040C9432040C9432040C94320468
:100040000C9432040C9432040C9432040C94320458
:100050000C9432040C9432040C9432040C94C32893
:100060000C9432040C94ED2B0C94232C0C9432043D
:100070000C9432040C9432040C9432040C94320428
:100080000C9432040C9432040C9432040C94320418
:100090000C9432040C9432040C9432040C94922785
:1000A0000C9432040C9432040C9432040C943204F8
:1000B0000C9432040C9432040C9432040C943204E8
:1000C0000C9432040C9432040C9432040C943204D8
:1000D0000C9432040C9432040C9432040C943204C8
:1000E0000C9432040C9432040C9432040C943204B8
:1000F0000C9432040C9432040C9432040C943204A8
:100100000C9432040C9432040C9432040C94320497
:100110000C9432040C9432040C9432040C94320487
:100120000C9432040C9432040C9432040C94320477
:100130000C943204E929EC29DB29DF29E529232A5B
:10014000F029F429FA29FE29022A082A0C2A102A61
:10015000232A162A1A2A1E2A0C946F160C94B813F6
:100160000C94082A0C945D260C94B02A0C94042B51
:100170000C94E2180C948A260C9488210C94EC2997
:100180000C94952A0C94E5290C94DB290C944D26AB
:100190000C94F4290C945B1B0C94CF250C94E02C4C
:1001A0000C9473040C94022A0C941A2A0C944D2C6F
:1001B0000C94B1250C94F0290C94D2090C94232AA8
:1001C0000C94DF290C94E91B0C94E9120C94A717EA
:1001D0000C94461D0C94D80D0C94932A0C94C125B4
:1001E0000C94FE290C9432260C94F5260C94162AB5
:1001F0000C94FA290C94C42A0C9465130C945C2674
:100200000C9438130C9411260C949A2C0C941E2ADE
:100210000C94A22A0C9432120C94102A0C94950778
:100220000C94262B0C94E9290C94E4090C94AB2132
:100230000C943A260C947C150C94572C0C944F1368
:100240000C94A90D0C94FF2C0C949A130C940C2A6A
:1002500000000000003E5B4F5B3E3E6B4F6B3E1C60
:100260003E7C3E1C183C7E3C181C577D571C1C5E77
:100270007F5E1C00183C1800FFE7C3E7FF0018244E
:100280001800FFE7DBE7FF30483A060E26297929F8
:1002900026407F050507407F05253F5A3CE73C5A2D
:1002A0007F3E1C1C08081C1C3E7F14227F22145F0A
:1002B0005F005F5F06097F017F006689956A606065
:1002C00060606094A2FFA29408047E040810207E5F
:1002D000201008082A1C08081C2A08081E101010E4
:1002E000100C1E0C1E0C30383E3830060E3E0E062A
:1002F000000000000000005F00000007000700147D
:100300007F147F14242A7F2A12231308646236493B
:100310005620500008070300001C22410000412223
:100320001C002A1C7F1C2A08083E08080080703028
:100330000008080808080000606000201008040297
:100340003E5149453E00427F40007249494946219D
:1003500041494D331814127F1027454545393C4A11
:100360004949314121110907364949493646494928
:10037000291E000014000000403400000008142270
:1003800041141414141400412214080201590906DE
:100390003E415D594E7C1211127C7F494949363EDF
:1003A000414141227F4141413E7F494949417F09C5
:1003B0000909013E414151737F0808087F00417FD0
:1003C00041002040413F017F081422417F404040CE
:1003D000407F021C027F7F0408107F3E4141413E66
:1003E0007F090909063E4151215E7F0919294626E8
:1003F0004949493203017F01033F4040403F1F20EC
:1004000040201F3F4038403F6314081463030478C2
:1004100004036159494D43007F41414102040810E2
:1004200020004141417F040201020440404040401D
:10043000000307080020545478407F28444438388B
:1004400044444428384444287F38545454180008FD
:100450007E090218A4A49C787F0804047800447DD7
:1004600040002040403D007F1028440000417F4074
:10047000007C047804787C080404783844444438C8
:10048000FC1824241818242418FC7C0804040848A8
:100490005454542404043F44243C4040207C1C20F9
:1004A00040201C3C4030403C44281028444C909054
:1004B000907C4464544C44000836410000007700AE
:1004C00000004136080002010204023C2623263CBB
:1004D0001EA1A161123A4040207A38545455592146
:1004E000555579412254547842215554784020542E
:1004F0005579400C1E52721239555555593954547C
:10050000545939555454580000457C410002457DEA
:10051000420001457C407D1211127DF0282528F013
:100520007C545545002054547C547C0A097F493240
:10053000494949323A4444443A324A4848303A41B7
:1005400041217A3A42402078009DA0A07D3D424260
:10055000423D3D4040403D3C24FF2424487E4943E9
:10056000662B2FFC2F2BFF0929F620C0887E09035C
:1005700020545479410000447D413048484A323883
:100580004040227A007A0A0A727D0D19317D2629AF
:10059000292F28262929292630484D4020380808A7
:1005A000080808080808382F10C8ACBA2F102834DB
:1005B000FA00007B000008142A142222142A1408CE
:1005C0005500550055AA55AA55AAFF55FF55FF00DD
:1005D0000000FF00101010FF00141414FF00101092
:1005E000FF00FF1010F010F0141414FC001414F7A6
:1005F00000FF0000FF00FF1414F404FC1414171093
:100600001F10101F101F1414141F00101010F000E2
:100610000000001F101010101F10101010F010001C
:100620000000FF101010101010101010FF1000002C
:1006300000FF140000FF00FF00001F10170000FC67
:1006400004F414141710171414F404F40000FF0039
:10065000F714141414141414F700F71414141714C2
:1006600010101F101F141414F4141010F010F000C8
:10067000001F101F0000001F14000000FC140000E9
:10068000F010F01010FF10FF141414FF14101010CD
:100690001F00000000F010FFFFFFFFFFF0F0F0F080
:1006A000F0FFFFFF0000000000FFFF0F0F0F0F0F14
:1006B0003844443844FC4A4A4A347E020206060260
:1006C0007E027E0263554941633844443C04407EC7
:1006D000201E2006027E020299A5E7A5991C2A4940
:1006E0002A1C4C7201724C304A4D4D3030487848CB
:1006F00030BC625A463D3E494949007E0101017EB7
:100700002A2A2A2A2A44445F444440514A44404009
:10071000444A51400000FF0103E080FF0000080848
:100720006B6B083612362436060F090F06000018C8
:10073000180000001010003040FF0101001F0101EF
:100740001E00191D1712003C3C3C3C00000000003C
:1007500000000000000000000007030401090A0B6C
:100760000000000200000000000000000000000087
:100770000000000001020408102040800110204009
:1007800080081020408004200102040810204080CE
:100790000204080102040102040404040404040421
:1007A0000202020202050505050505070606060602
:1007B00006060606020202070707050500000000FC
:1007C000250000002B002E00310034000000000046
:1007D00000000000000000000000240000002A00CB
:1007E0002D00300033000000000000000000000079
:1007F0008821B125C1251126F526572CE02CAB21E7
:10080000CF2511241FBECFEFD1E8DEBFCDBF00E062
:100810000CBF15E0A0E0B2E0E2E9F8E600E00BBFB3
:1008200002C007900D92A43DB107D9F72FE0A4EDC7
:10083000B5E001C01D92A031B207E1F717E0CEEF9D
:10084000D7E000E006C022970109FE010BBF0E941D
:10085000BE30C03FD10780E00807A9F70E94F02C06
:100860000C9437340C9400001092D80E1092D90ECC
:100870001092D50E1092D40E10920B0F10920A0FF8
:10088000EAEDFEE0119211928EE0EA3FF807D1F70F
:100890000E940F0E0E94050A0E9453050E948F04B9
:1008A0000E94C3050E946A0C0C949B089093D50E7D
:1008B0008093D40E0C9411109093D70E8093D60E83
:1008C0000C94FF0FE82FF0E0EE0FFF1FE652F14F00
:1008D0007183608308950E945E0A0E942D0F0E941A
:1008E000B2040C94B80CE091D405F091D505309782
:1008F000A1F0228133812817390759F4DC01AD5763
:10090000BF4F2C91278713962C91208B22E02483B4
:1009100004C00190F081E02DEACF0C948F05109275
:10092000D5051092D4050895FC0114821786138210
:10093000128280910A0F90910B0F019690930B0FEA
:1009400080930A0F8091D4059091D505009719F4F2
:100950001182108202C091838083F093D505E093C9
:10096000D40508950F931F93CF93DF93E091D4059F
:10097000F091D505EF01209709F490C08C81882370
:1009800021F0823009F460C085C00E945E058C01B0
:10099000009721F482E08C838F8780C09B838A83B9
:1009A00081E08C83F801E957FF4F83E794E091835E
:1009B00080833197898582FB882780F98083998598
:1009C000F801838590FB80F98387998593FB9927AC
:1009D00090F990FB82F9838799859695917090FBA9
:1009E00081F983878091D80E8F5F8093D80E84879A
:1009F0008091D40E9091D50E968785878D819E81AA
:100A0000908B878798859F708189807F892B818BC8
:100A10009F819295907F8F70892B818BEF57FF4F2D
:100A20004C8550E06A857B85808191810E946E3380
:100A3000F80181819C85890F8183C801DF91CF9165
:100A40001F910F910C94400EEC17FD0739F488812B
:100A500099819093D5058093D4050BC080819181B5
:100A60008C179D0711F0FC01F9CF88819981918342
:100A7000808380910A0F90910B0F019790930B0F39
:100A800080930A0FED85FE85CE01DF91CF911F91F6
:100A90000F9119940990D881C02D6DCFDF91CF911E
:100AA0001F910F9108951092D60510925F06109233
:100AB000E806109271071092FA070895E6EDF5E046
:100AC00080E090E02081211121C049E8489F9001F9
:100AD000499F300D1124C9018A529A4FFC0111928D
:100AE0004A95E9F740E1FC014183EF57FF4F285158
:100AF0003A4F3183208320910A0F30910B0F2F5FE3
:100B00003F4F30930B0F20930A0F08950196E7573C
:100B1000FF4F85309105B1F680E090E00895FC012B
:100B20001082EAE0FFE080819181019791838083C8
:100B30000895009711F0FC0103C0E6EDF5E002C056
:100B4000E757FF4F88E0E338F80728F480818823CF
:100B5000B9F3CF01089580E090E00895FC01DC0135
:100B6000AD57BF4F1C92A8EDBEE08C918F5F8C9368
:100B700084878091D40E9091D50E96878587838542
:100B8000826083870895E8E8F8E080E090E02FEF46
:100B90003FEF57E0DF0114972D933C93589FD0010E
:100BA000599FB00D1124AD57B74F4C914E7F4C93C8
:100BB0001082019637968431910561F70895CF939D
:100BC000DF93A4E8B8E020E030E0C7E070E0ED910A
:100BD000FC911197E817F90789F4C29FF001C39FB0
:100BE000F00D1124ED57F74FD081D1FB442740F988
:100BF00050E04617570711F4CF0108C02F5F3F4F51
:100C000017962431310519F780E090E0DF91CF91FC
:100C10000895E0E0F0E0A3E8B8E08C9180FD0BC01F
:100C200015968C911597882361F0309719F095816E
:100C3000891708F4FD01179689E0AF30B80769F706
:100C400001C0FD0180818D708063808380E8858391
:100C5000CF010895FC01808180FD05C08FEF9FEFDB
:100C600092838183158208950E94DF05009721F009
:100C7000FC018381948108958FEF9FEF089583E8AD
:100C800098E00895EF92FF920F931F93CF93DF9315
:100C9000EC01F62E8A01E22E0E94DF05FC0100978E
:100CA00019F40E940906FC01D283C18314830383D3
:100CB0008081F0FA81F98F708063808380E885837A
:100CC000E682DF91CF911F910F91FF90EF900895F1
:100CD0000E94DF05009711F00C942A0608950895EC
:100CE000CF93DF93EC018F8598898F3F2FEF920789
:100CF000B1F16B8563FB662760F90E94DF05FC019B
:100D0000009769F1808180FD2AC0CD57DF4F98811F
:100D1000282F2F70911113C02063208385818F5F4E
:100D200085838F3FE1F4E8E8F8E0808186958F5F66
:100D30008083379689E0E431F807B9F710C08295CF
:100D40008F70815F8F70982F9295907F922B9083F8
:100D5000811105C0CF01DF91CF910C942A06DF915C
:100D6000CF910895CF93DF93EC018F8598898F3FC2
:100D70002FEF920719F06B8562FF03C098878F836E
:100D80000EC063FB662760F90E94340698878F8344
:100D9000019629F4CE01DF91CF910C94C608DF9122
:100DA000CF910895BF92CF92DF92EF92FF920F936F
:100DB0001F93CF93DF938C01FC01B384B3FABB2460
:100DC000B0F8C784D0886B2DC6010E943406019606
:100DD000A1F0F801E957FF4F11821082319782E0AC
:100DE0008083C801DF91CF911F910F91FF90EF9009
:100DF000DF90CF90BF900C94400EF801E584F6840C
:100E00000E945E05EC010097D1F00E94AE05898139
:100E10008A5F8983FE01E957FF4F11821082F88AA9
:100E2000EF8636970190F081E02D81E08083F28299
:100E3000E182D482C382B582CE010E94400EC801F5
:100E4000DF91CF911F910F91FF90EF90DF90CF90A6
:100E5000BF900C948F05DC011796ED91FC911897CB
:100E600019968C91863039F46581838194810E9432
:100E7000680681E0089580E00895CF93DF93EDE167
:100E8000F9E0A1E2B9E020E030E0C185D285CD2BC8
:100E9000B1F0C081D181C817D90789F4C281D3814B
:100EA000C617D70761F45C91541309C04BE0429F09
:100EB000C001439F900D1124835E964F09C02F5FA0
:100EC0003F4F3B961B9625303105F9F680E090E0C8
:100ED000DF91CF910895CF93DF93E6E2F9E080E0D0
:100EE00090E020813181232BA9F42BE0289FE001A1
:100EF000299FD00D1124C35ED64F209791F01F82F9
:100F0000188688EE93E09A8789878FE099E00E949F
:100F1000D11107C001963B968530910511F7C0E0CD
:100F2000D0E0CE01DF91CF9108958F929F92AF9242
:100F3000BF92CF92DF92EF92FF920F931F93CF93C6
:100F4000DF935C010DE119E0E12CF12C912CF8010B
:100F5000218532852536310538F02456310932870E
:100F600021879924939438C0F80112861186208134
:100F700031818091D40E9091D50E2817390761F5F3
:100F8000C701835E964F6C01FC018084C0E0D0E015
:100F9000CE010E949905EC010097F1F08881803420
:100FA000B9F7F801228133818F859889281739078D
:100FB00079F78B8583FB882780F9F6019481981354
:100FC000E7CF882021F0CE010E94400EE1CF61E101
:100FD000CE010E94010FDCCFFBE0EF0EF11C055F9C
:100FE0001F4F87E3E816F10409F0B1CF992079F09B
:100FF000C501DF91CF911F910F91FF90EF90DF908E
:10100000CF90BF90AF909F908F900C94D111DF91B3
:10101000CF911F910F91FF90EF90DF90CF90BF90F5
:10102000AF909F908F900895FF920F931F93CF934F
:10103000DF938C01F62E0E945E05EC01009761F1B2
:101040000E94AE058981895F8983FE01E957FF4FC0
:10105000118210828B8584608B878FEF9FEF988B36
:101060008F8736970190F081E02D82E08083D80150
:101070008D919C9111979283818312968D919C9171
:1010800013979483838314968C918583F682CE0183
:101090000E94400E81E001C080E0DF91CF911F915E
:1010A0000F91FF900895EF92FF920F931F93CF93AC
:1010B000DF938C01E62EF42E0E945E05EC01009772
:1010C00099F10E94AE058981885F8983FE01E95705
:1010D000FF4F11821082319784E08083D8011596EA
:1010E0008D919C911697988B8F8735970190F08101
:1010F000E02D83E080838D919C9111979283818371
:1011000012968D919C9113979483838314968C915E
:101110008583E682F782CE01DF91CF911F910F91F7
:10112000FF90EF900C94400EDF91CF911F910F91A3
:10113000FF90EF90089510922709109226091092BF
:1011400032091092310910923D0910923C09109217
:10115000480910924709109253091092520984E6E7
:1011600090E0A0E0B0E08093150990931609A09359
:101170001709B093180910921A091092190985E9F4
:1011800097E090931C0980931B090895CF93DF93F8
:10119000EC014B8543FB442740F96F8578898091AA
:1011A000D40E9091D50E0E943D07892BE9F40E9440
:1011B0006B070097F1F02091D40E3091D50EFC0111
:1011C000318320832F853889338322832B8523FB2A
:1011D000222720F924832FEF3FEF368325836FEFFB
:1011E0000E941408882329F080E48883DF91CF913E
:1011F000089561E1CE01DF91CF910C94010FAF9280
:10120000BF92CF92DF92EF92FF920F931F93CF93F3
:10121000DF936C01FC01078110858185873009F01F
:101220005AC0F80145812091D40E3091D50E41115C
:1012300007C0BB24B394838194818217930709F07C
:10124000B12CF801818192818217930709F441C082
:10125000B11002C037FD3DC0F601E284F8012681DD
:10126000E29E70011124638174810E943D07EC01AC
:10127000009721F08F818F1530F02BC00E946B07F3
:10128000EC01009731F1F801818192819983888383
:10129000838194819B838A8385818C83F6018081FD
:1012A00091819E838D83FF82BB2079F040815181A3
:1012B0002F2D60E0F801818192810E9442064FEF5C
:1012C0006F2DCE010E94530804C06F2DCE010E94E5
:1012D000140881E001C080E0DF91CF911F910F9150
:1012E000FF90EF90DF90CF90BF90AF900895EF9276
:1012F000FF920F931F93CF93DF937C01DC0117962E
:10130000CD91DC91189719968C91883009F040C0E6
:101310006B817C814D8189819A810E943D078C017E
:10132000D7011A96FC91EF810097A1F18E81D80127
:1013300018969C911897981768F518968C93698160
:101340007A812091D40E3091D50E8B819C81D7016A
:101350004D915C916217730729F42E816D810E9473
:10136000420618C0FE9F700111242F2D6D810E942E
:101370004206F80145815681278160E089819A8182
:101380000E9442064F2D6E81C8010E94530802C080
:1013900080E001C081E0DF91CF911F910F91FF901C
:1013A000EF900895E7E6F9E020E03081332319F06B
:1013B0003150308321E035963AE0E136F307A9F762
:1013C00021110C94D1110895DC0116962C911697D9
:1013D00021FF19C019962C9119972223A1F0179675
:1013E000ED91FC9118972081213049F030F02230A6
:1013F00041F0233041F40C9477090C94DF0E0C94E7
:101400002B070C94FF0880E00895E7E6F9E01082CE
:1014100035968AE0E136F807D1F784E690E0A0E05F
:10142000B0E080935A0990935B09A0935C09B09354
:101430005D0910925F0910925E0982ED99E0909328
:1014400061098093600964EE79E080E00C946204A5
:10145000CF93DF93EC01E881F9818181883801F530
:1014600080818F7D8134E1F48A818031C8F00E94CF
:101470005E050097A9F020E2FC0120832A812183E8
:101480002B81ED57FF4F20832C81319620834A8199
:1014900050E0688179810296DF91CF910C946E3390
:1014A000DF91CF910895809362090895662311F02A
:1014B00022E201C024E2FC01208308956F927F9212
:1014C0008F929F92AF92BF92CF92DF92EF92FF9254
:1014D0000F931F93CF93DF93CDB7DEB72C970FB643
:1014E000F894DEBF0FBECDBF00E010E094E2D92E2D
:1014F0008824839422E2C22E31E2B32E43E2942E5A
:1015000052E0A52EEE24E394F12CC8010E94990527
:101510008C01009709F4C9C1D8018C91823209F479
:10152000B6C048F4803281F0813279F760E0C801BA
:101530000E94710CEACF833209F47CC1843229F70E
:10154000C8010E948F05E1CFF801D082438543FD99
:10155000DCCF25813681878590892F3F3F4F89F4E5
:101560002091D40E3091D50E2817390711F001962D
:1015700061F641FF03C0D801BC92C7CFF801C08219
:10158000C4CF019611F440FDC0CF2091D40E30910C
:10159000D50ED8011D968D919C911E97281739075D
:1015A00009F4B3CFC8010E946F06E3E6F9E040E01A
:1015B00050E08481882309F44AC0D8011D962D91FA
:1015C0003C911E97808191812817390709F040C00E
:1015D0001C969C911C974281491B8381483060F581
:1015E000282F30E0042E02C0359527950A94E2F7A3
:1015F00020FF19C02091D40E3091D50E17968D91F1
:101600009C9118972817390709F07FCF1B966C918A
:101610001B9763FB662760F91F968D919C915097ED
:101620000E94680672CF9701042E01C0220F0A940F
:10163000EAF7822B838302C192834195042E01C075
:10164000880F0A94EAF781608383A482F7C0AF0110
:101650003596BAE0ED35FB0709F0ABCF41155105E2
:1016600009F453CFF80185859685DA0111969C938C
:101670008E93848512968C93129713968C9213975F
:101680001496AC9284E599E00E94D111D7C01092D3
:101690006209D80151963C915197232F22952F70C2
:1016A000E22FF0E0EE0FFF1FE652F14F0190F081C4
:1016B000E02D309709F45DC01D968D919C911E9789
:1016C0009A8389831F964D915C9150975C834B83DD
:1016D0003F703D832E83AF57BF4F6D917C917987CB
:1016E000688798012E5F3F4F261B370BD801119654
:1016F0003C911197320F3A87AD57BF4F2C912B87F2
:1017000011962C912C87D8011B962C91622F637017
:1017100022FF02C030E201C030E0632B23FF02C091
:1017200030E401C030E0362B4F3F5F4F11F424E02E
:1017300001C020E0432F422BD80119962D913C91F6
:101740001A978217930711F498E001C090E0242FB4
:10175000292BD80115968D919C911697019611F41D
:1017600080E101C080E0822B8F83CE010196199524
:1017700001C080E0F801938590FF80E0D8011796C2
:101780004D915C9118972091D40E3091D50E4F3F1A
:101790005F4F41F4F801478550892417350711F44C
:1017A00093FF81E0D80115964D915C9116974F3FBC
:1017B0005F4F09F480E02F3F3F4FC9F18823B9F113
:1017C0000E945E053C01009791F10E94AE05D30195
:1017D00011968C9111978D5F11968C931197F3014F
:1017E000E957FF4F11821082F80193859695917009
:1017F0001B968C911B9790FB81F91B968C931B97E2
:101800008585968550969C938E931F97F301EF578D
:10181000FF4F0190F081E02D108280916209828358
:10182000D8011C968C918183C3010E94400EF8015F
:10183000D0826BCEC8010E94D20667CED80117961F
:101840008D919C911897019681F42091D40E30913E
:10185000D50EF801878590892817390731F08385DF
:1018600082FD03C0C8010E94970E8091D40E909112
:10187000D50ED8011F962D913C915097F8018217F3
:10188000930719F02F3F3F4F41F4838581FF02C03A
:10189000B0823BCED801CC9238CE278130858217DA
:1018A000930709F032CE908230CE2C960FB6F89482
:1018B000DEBF0FBECDBFDF91CF911F910F91FF9083
:1018C000EF90DF90CF90BF90AF909F908F907F90E0
:1018D0006F9008951092720A1092710A1092700A15
:1018E0000895662311F020E301C021E3FC01208369
:1018F0008091720A8F5F8093720A0895CF93DF936D
:10190000C091700AD091710A60916E0A40916F0A7D
:10191000342F413108F030E170916D0A8DE59AE085
:10192000FE01EF57FF4FA081B181A60FB11DFC0151
:101930002E2F281B231768F420815C9125272D93D7
:10194000772311F0208303C05081522750833196B2
:10195000EFCF630F60936E0A431B40936F0A4423DB
:1019600011F082E301C084E38883DF91CF91089571
:101970000F931F938091720A882309F4E7C0809126
:10198000700A9091710A009709F46FC0FC012081E0
:10199000243309F05CC020916E0AEF57FF4F01908D
:1019A000F081E02DE20FF11D4091610A5091620A31
:1019B0006091630A7091640A00915D0A10915E0A59
:1019C00020915F0A3091600A4027512762277327D0
:1019D0000091650A1091660A2091670A3091680AA1
:1019E00040275127622773270091690A10916A0ADC
:1019F00020916B0A30916C0A402751276227732788
:101A000020916D0A222359F04083518362837383AE
:101A1000FC0121812C5F21830E94080F0EC0A1E0F0
:101A200000811181228133814017510762077307BA
:101A300009F0A0E06A2F0E94560A1092710A1092D3
:101A4000700A8091720A81508093720A7FC022339B
:101A500009F07CC023E3FC0120836AEF7EE08DE582
:101A60009AE01F910F910C945B11E0E0F0E0CF0140
:101A70000E949905FC01009709F468C0808190EDEF
:101A8000980F9230A0F7F093710AE093700A4485A2
:101A900050E060E070E040935D0A50935E0A60930E
:101AA0005F0A7093600A4785508960E070E0BA0170
:101AB00055274427918992959F70492B4093610A3D
:101AC0005093620A6093630A7093640A4585568551
:101AD00060E070E0BA015527442791899F70492B37
:101AE0004093650A5093660A6093670A7093680A88
:101AF00093854581568160E070E0BA0155274427FF
:101B0000492B4093690A50936A0A60936B0A709359
:101B10006C0A813319F49181945091839F012E5F57
:101B20003F4FDF01AF57BF4F4D915C91241B350BE9
:101B30009181920F90936F0A10926E0A91E0803318
:101B400009F090E090936D0A82E380831F910F91DA
:101B500008950F931F93CF93DF93EC0110E0E0E023
:101B6000F0E003E1CF010E949905FC01009791F09C
:101B700080818131B9F7DF01AC57BF4F2D913C9186
:101B80001197215031092D933C93232B09F40083A5
:101B900011E0E8CF112339F0CE01DF91CF911F91F1
:101BA0000F910C94D111DF91CF911F910F91089556
:101BB000FF920F931F93CF93DF93EC0110E0E0E0CF
:101BC000F0E007E180E1F82ECF010E949905FC01C9
:101BD0000097A9F080818631B9F7DF01AC57BF4F7C
:101BE0002D913C9111972150310911963C932E93E0
:101BF000232B19F400831197FC9211E0E5CF1123F8
:101C000041F0CE01DF91CF911F910F91FF900C9485
:101C1000D111DF91CF911F910F91FF9008951092F4
:101C2000900A10928F0A82E390E0A0E0B0E08093E7
:101C3000870A9093880AA093890AB0938A0A10921F
:101C40008C0A10928B0A88ED9DE090938E0A809307
:101C50008D0A8AE090E0A0E0B0E08093790A90934A
:101C60007A0AA0937B0AB0937C0A10927E0A1092A3
:101C70007D0A89EA9DE09093800A80937F0A089507
:101C80000F931F93CF93DF93EC01FC01EA57FF4FB3
:101C9000208121FF02C082E104C08B8581FFFBCF40
:101CA00080E18883FE01ED57FF4F108220FF03C0C3
:101CB0008FEF9FEF04C08091D60E9091D70E9E8338
:101CC0008D83257021F4CE010E94B20604C08F8559
:101CD000988998878F838091D40E9091D50E9A879A
:101CE00089878091D90E8F5F8093D90E8C838F81E5
:101CF00098858E010C571F4F019669F481E498E88E
:101D00009B838A830E944A32877099270196F80143
:101D10009183808307C081E698E89B838A83F801DA
:101D200011821082DF91CF911F910F9108950F932F
:101D30001F93CF93DF938C010E945E05EC01009707
:101D4000C9F182E18883F80181818983FE01ED5721
:101D5000FF4F10820E944A32FE01EC57FF4F8770FE
:101D60009927019691838083339611821082F8011E
:101D7000418150E0B8016E5F7F4FCE0102960E9414
:101D80006E3381E498E89B838A838FEF9FEF988777
:101D90008F83F801858196819E838D838091D40EF7
:101DA0009091D50E9A8789878091D90E8F5F809305
:101DB000D90E8C83DF91CF911F910F910895CF930E
:101DC000DF93FC01C781D0858185833011F080E0ED
:101DD00015C080E090E00E9499050097C1F3FC01D6
:101DE00020812631C1F7348529813213F4CF27E1D0
:101DF00020832A81EA57FF4F208381E0DF91CF9132
:101E0000089527E1FC012083ED57FF4F608308957B
:101E100022E1FC0120830895A0918F0AB091900ADD
:101E2000833030F4E82FF0E0E65EFB4F808101C0A4
:101E300081E0FD01ED57FF4F808385E18C93109287
:101E4000900A10928F0A80910A0F90910B0F0197C0
:101E500090930B0F80930A0F0895BF92CF92DF9259
:101E6000EF92FF920F931F93CF93DF93C0E0D0E0E8
:101E700094E1E92E27E1F22E36E1D32E05E010E0C1
:101E800043E1C42E51E1B52ECE010E949905EC012B
:101E9000009709F469C088818331F1F028F480311A
:101EA00049F0823161F0F0CF853181F1873109F459
:101EB0004AC0EACF61E0CE010E94710CE5CFFE017D
:101EC000EC57FF4F80819181892B21F0B88283E705
:101ED0009AE034C0C882D8CF80918F0A9091900A3E
:101EE000892B91F6D093900AC0938F0AE88269817A
:101EF000CE0102960E942B1080910A0F90910B0F39
:101F0000019690930B0F80930A0FBECFFE01ED5701
:101F1000FF4F8081811115C02D853E858091D40EA3
:101F20009091D50E2817390761F48B8580FF09C081
:101F3000D88231961183008381E89AE00E94D11102
:101F4000A3CFF882A1CFCE010E947006FE01E9570F
:101F5000FF4F0190F081E02DCE01309719F40E94DF
:101F60008F0592CF199590CFDF91CF911F910F914F
:101F7000FF90EF90DF90CF90BF9008959091910ADD
:101F80009F7080915401807F892B809354019091A0
:101F9000910A8091920A992319F080935301089530
:101FA000982F9F7180914801807E892B80934801F2
:101FB000089593E090934201909141019F71983070
:101FC000D9F780934201909141019F718913FBCF12
:101FD000089588E00E94D90F8FEF80934F01809180
:101FE000930A882319F086E10C94D90F0895809301
:101FF000930A0C94E90F8093920A0C94BE0FCF932E
:10200000DF931F921F92CDB7DEB79A8389838093A7
:1020100062018A81809363010F900F90DF91CF91CD
:102020000895CF93DF931F921F92CDB7DEB79A83A7
:102030008983809360018A81809361010F900F9062
:10204000DF91CF9108958F70E5E4F1E09081907F6A
:10205000982B908308951F93CF93DF931F921F9225
:10206000CDB7DEB7182F89E169839A830E94D90F13
:102070008FEF80934F01698182E0860F809380010A
:10208000212FE12F9A81F92FA1E8B1E08E2F821B39
:10209000861718F481918D93F9CF83E090E09093A7
:1020A000150B8093140B82E0809342010F900F90E8
:1020B000DF91CF911F9108950F931F93CF93DF93DB
:1020C0001092560186E00E94D90FC0E0D0E000E0F7
:1020D00010E061E070E080E090E00E943C29809197
:1020E000460182958695837090E00C2E02C0880F81
:1020F000991F0A94E2F7082B192B2296C031D105BB
:1021000041F788E00E94D90F8BEE809356010E9420
:10211000E90FC801DF91CF911F910F910895E9E375
:10212000F1E08081816080831092930A1092910A7D
:1021300081E090E09093150B8093140B88E00E944F
:10214000D90F8BEE80935601ECE4F1E0808180683A
:1021500080830E945C1080936D01089520E1FB0153
:102160003191BF0130933F012150C9F710923C01DA
:10217000FC0120E1319130933E012150D9F72091AB
:102180003C01206820933C0120913D0120FFFCCFC1
:10219000FC0180E190913E0191938150D9F708951F
:1021A000CF93DF9300D000D0CDB7DEB78091140B72
:1021B0009091150B029709F469C080914F0183FF3C
:1021C0003CC050917B0140E0252F30E0842F90E00F
:1021D0002817390754F0FC01E058FE4F6081FC01DC
:1021E000EC56F54F60834F5FF1CF84E99AE09A8314
:1021F000898352505B83F901EC56F54F80818C83C3
:10220000809147018F5F8D83CE0101960E94280A3D
:10221000809141018F718631D9F780914F0188609B
:1022200080934F0180914C018F7780934C01809176
:102230004C01806880934C0129C080914F0186FF3A
:1022400025C0809141018F718931D9F4809142017B
:1022500082958695877049F0833021F0853021F48E
:1022600082E003C081E001C083E08E830E94E90F19
:1022700021E030E03093150B2093140B8E810E94E7
:102280000C0F80914F01806480934F0126960FB60A
:10229000F894DEBF0FBECDBFDF91CF9108950E94AD
:1022A000BB110E948F100C9434040E94D0100E9425
:1022B0006B040C94E0110E94AE100C947E0C0F93F2
:1022C0001F93CF93DF93FC018091170B9091180B14
:1022D000B681A781308521850097F1F14B2F5A2FC8
:1022E000632F722FDC01D0E0C0E012960D911D919A
:1022F0002D913C911597401751076207730768F4B9
:10230000041B150B260B370B12960D931D932D9363
:102310003C931597AD2FBC2F0EC0401B510B620B89
:10232000730B2D913C9111972115310521F0DA2F76
:10233000CB2FD901DACF42835383648375831097FF
:1023400041F08D919C91119791838083ED93FC9343
:102350000DC09183808306C011821082B283A38353
:1023600034832583F093180BE093170BDF91CF9103
:102370001F910F9108951092180B1092170B08954A
:10238000E091170BF091180B309739F0E817F90727
:1023900031F00190F081E02DF7CF80E0089581E0E9
:1023A0000895CF93DF93EC010E94C011811105C005
:1023B000CE01DF91CF910C945F11DF91CF91089501
:1023C000CF92DF92EF92FF92CF93DF930E940D297D
:1023D0002091160BC22ED12CE12CF12C6C157D0511
:1023E0008E059F05C1F10E940D298091160BC62E06
:1023F000C81AD12CE12CF12C6093160BC091170B4D
:10240000D091180B209739F14A815B816C817D81D5
:10241000C416D506E606F706B0F0C41AD50AE60AD1
:10242000F70A888199819093180B8093170B8A85FE
:102430009B85019719F4CE010E945F11EC85FD8503
:10244000CE011995DBCF4C195D096E097F094A83CE
:102450005B836C837D83DF91CF91FF90EF90DF9062
:10246000CF9008952F923F924F925F926F927F92FA
:102470008F929F92AF92BF92CF92DF92EF92FF9294
:102480000F931F93CF93DF9300D01F92CDB7DEB78A
:102490004C017C836B836A015901C8018701AC013F
:1024A0004C195D0957FF03C051954195510995019C
:1024B0006B817C81261B370B37FF03C0319521953B
:1024C000310922242394312C2417350714F0212CB0
:1024D000312C2114310459F03A2D2B2D5C01832F1E
:1024E000922F3B812C81DC82CB82C32ED22EAB81FA
:1024F000BC81AA16BB065CF43C2D2D2D6C01832FEC
:10250000922F3B812C81BC82AB82A32EB22E25015F
:10251000EB81FC814E1A5F0A3C016C187D0877FE46
:1025200003C0719461947108720157FE03C0FFEFFC
:10253000EF1AFF0AF594E794C816D9062CF421E0A7
:1025400030E03A83298324C06FEF7FEF7A83698379
:102550001FC0D401ED91FC910480F581E02D98011C
:1025600021143104D9F04B815C81B601C401199565
:10257000E618F708F7FE06C0E981FA81CE0EDF1EE5
:10258000E40CF51C2B813C812F5F3F4F3C832B8358
:102590006B817C81A616B706E4F604C0A6016B81A8
:1025A0007C81E4CF0F900F900F900F90DF91CF912F
:1025B0001F910F91FF90EF90DF90CF90BF90AF9061
:1025C0009F908F907F906F905F904F903F902F9053
:1025D00008956F927F928F929F92AF92BF92CF9207
:1025E000DF92EF92FF920F931F93CF93DF93EC0153
:1025F0005B016A0139014801E881F9810284F385B0
:10260000E02D87011995E881F981A601480D591D32
:10261000415051090284F385E02D9301B501CE01AB
:102620001995E881F9810084F185E02D9401A601D6
:10263000B501CE011995E881F981B501660D771DC7
:10264000615071090084F185E02D9401A601CE014D
:102650001995DF91CF911F910F91FF90EF90DF902F
:10266000CF90BF90AF909F908F907F906F90089584
:10267000EF92FF920F931F93DC01ED91FC91240FD9
:10268000351F215031090680F781E02D780189013D
:102690009B0119951F910F91FF90EF900895EF9274
:1026A000FF920F931F93DC01ED91FC91260F371FD2
:1026B000215031090680F781E02D78018A011995B2
:1026C0001F910F91FF90EF9008956F927F928F92DC
:1026D0009F92AF92BF92CF92DF92EF92FF920F93B1
:1026E0001F93CF93DF935C014A0169013801EB012D
:1026F000C60ED71ECC15DD0574F4D501ED91FC9105
:102700000084F185E02D87019301A401BE01C5017C
:1027100019952196EFCFDF91CF911F910F91FF90E7
:10272000EF90DF90CF90BF90AF909F908F907F9071
:102730006F900895EF92FF920F931F93DC01ED913C
:10274000FC9111971A960D911C911B9718962D913B
:102750003C9119970684F785E02D7B0140E050E01D
:1027600060E070E019951F910F91FF90EF90089530
:102770000895FC011382128281E294E091838083A8
:102780007583648357834683718760875387428745
:10279000158A158614861786168621E0248B8FEFFE
:1027A0009FEF938B828B918B808B268B178A118E58
:1027B000108E08952F923F924F925F926F927F9268
:1027C0008F929F92AF92BF92CF92DF92EF92FF9241
:1027D0000F931F93CF93DF93CDB7DEB76A970FB6F2
:1027E000F894DEBF0FBECDBF1C0158874F831C87F6
:1027F0000B87FA86E986CC82DC0158964D915C9174
:1028000059974115510509F0A6C018968D919C91D4
:102810001997681779070CF056C11A968D919C91FB
:102820001B97EF81F885E817F9070CF04CC1D12C04
:10283000CB013C81F6E03F9F800D911D11241816BD
:1028400019060CF040C1C60103E0880F991F0A95D4
:10285000E1F74F815885840F951F181619060CF063
:1028600032C157968C91811103C0203B08F02F5F35
:102870007E876D874B01198210E5A12E12E0B12EE3
:10288000A61AB70A55E0259FA00CB11C1124898116
:10289000853039F0ED85FE85EA0DFB1D94919A8314
:1028A00001C01A826F8078842301A8E0AD83BA81C9
:1028B000B0FF12C0D101ED91FC91BC81B13031F477
:1028C0000480F581E02D2B853C8518C00684F785B2
:1028D000E02DEB84FC841DC0E985FA852B853C85C1
:1028E000E217F307E1F0D101ED91FC91BC81B13029
:1028F00059F40480F581E02D29853A85A2016D8582
:102900007E85C10119950BC00684F785E02DE98409
:10291000FA8486019601A301B401C1011995EA81E7
:10292000E695EA83FD81F150FD836C0C7D1C2FEF51
:10293000421A520AF111BBCF39813F5F39838C0CA7
:102940009D1C4D855E854F5F5F4F5E874D8736309E
:1029500009F09DCFB8C0FA01349634913297859131
:102960009491231BA7E02A9F800D911D1124FA0149
:1029700025913491398B288BFC01459154915A8FC4
:10298000498FFC013296549159873196A491AF87B3
:102990003196E491FC013596249131968491BC8165
:1029A000B23050F0622E772467FC7094E82FFF2736
:1029B000E7FDF095FE87ED87FC81CF2ED12C6C9C36
:1029C00040016D9C900C7C9C900C1124860E971EEF
:1029D000A12C1982DE8ACD8AAB01420F511D27FD41
:1029E0005A955E834D83AF81B885A80FB11D87FDD1
:1029F000BA95B88FAF8B59818F85581708F063C08F
:102A0000852F90E02D853E85280F391F2C9DD00104
:102A10002D9DB00D3C9DB00D1124EF81F885EA0F7E
:102A2000FB1FFB83EA836D807E802401FA2D2D81BC
:102A3000F21BFA8B4F89588D480F591F5C8B4B8BBB
:102A40009A89960D862D2D81821B39858317B0F5C5
:102A5000977061F4898D9A8D0196E889F989298D9D
:102A60003A8DE20FF31FB4909A8F898FB7FE1DC085
:102A7000D101ED91FC91BC81B13059F40480F58114
:102A8000E02D2B853C854B895C89B301C1011995EB
:102A90000CC00684F785E02DEB84FC84860196014A
:102AA0004A815B81B201C1011995BB0CED89FE8998
:102AB0004E0E5F1EFFEF6F1A7F0AC2CFA30E498131
:102AC0004F5F498398CF6A960FB6F894DEBF0FBE6A
:102AD000CDBFDF91CF911F910F91FF90EF90DF90CD
:102AE000CF90BF90AF909F908F907F906F905F90AE
:102AF0004F903F902F900895AF92BF92CF92EF9258
:102B0000FF920F931F93CF93DF93EC01262F888DB5
:102B1000998D009709F042C06A3069F42C898E853E
:102B20009F8538E0239F800D911D11249F878E87FC
:102B30001D861C86ABC06D3009F4A8C08E89882321
:102B4000C1F03C898C859D8546E0349F800D911DA8
:102B5000112448855985841795075CF01D861C86CD
:102B60008E859F85E8E03E9F800D911D11249F87F3
:102B70008E87EA88FB88088919894E855F856C8570
:102B80007D85CC88CE010E94DA132C898C859D85A9
:102B9000F6E02F9F800D911D112441C06A3079F419
:102BA0001D861C864C89FC01369684912E853F85B6
:102BB000489F200D311D11243F872E8767C06D303F
:102BC00009F464C0AC014C5F5F4FFA0134916317A4
:102BD00008F45CC03196E491E61708F457C0FA0196
:102BE0004491362F341BFC013296A590B490F7E047
:102BF0003F9FA00CB11C1124F5013296A49131968F
:102C0000E491AA2311F0E1110DC0F5013496A490CE
:102C10002C898C859D85A29E800D911D11249D87F8
:102C20008C8734C0F5013596E4913E89332309F150
:102C30003C89B0E0AE0FB11DE7FDBA953A9FA00107
:102C40003B9F500D11246C857D85460F571F68856D
:102C50007985461757076CF01D861C86FC01369651
:102C600084914E855F85389F400D511D11245F87EB
:102C70004E87EA88FB88088919894E855F856C85AF
:102C80007D85CC88CE010E94DA13BFCF81E090E031
:102C9000DF91CF911F910F91FF90EF90CF90BF9058
:102CA000AF900895FC01758764875787468708951C
:102CB000611101C061E0FC01648B0895FC01738B1C
:102CC000628B718B608B0895FC0185890895FC01EE
:102CD000808591850895FC018285938508950F93E1
:102CE0001F93CF93DF93EC018D89823061F08330A5
:102CF000D9F0813009F0C8C0EC81FD81E41BF50BEF
:102D00003197DB0118C08C819D81DC01A61BB70BBC
:102D1000BD018E819F81FC01E41BF50BAF01415089
:102D20005109621B730BB0C0AE81BF81A61BB70BEC
:102D3000A21BB30BFA01F7FD05C18C819D81E81739
:102D4000F9070CF0FFC0B7FF04C02A0F3B1FA0E03B
:102D5000B0E08E819F81AD01420F531F841795070C
:102D60001CF49C012A1B3B0B121613060CF0EAC044
:102D7000422F8A2F86958695869590E8899FE00D4B
:102D8000F11D1124E65EFD4FA77069F158E05A1B52
:102D9000852F90E0EC01CE5EDD4F6881251760F451
:102DA000DC01A21BB1098FEF90E00A2E02C09595BD
:102DB00087950A94E2F768230130110539F048F04D
:102DC0000230110551F48081862706C08081862B50
:102DD00003C06095808186238083451708F4B2C0C4
:102DE000451BE058FF4F4830A0F102301105A9F40F
:102DF000DF01842F9C9190959C93A058BF4F8850E1
:102E00008830C0F788EF840F869586958695B0E860
:102E10008B9FE00DF11D112419C081E001301105D7
:102E200009F080E0982F9195EF01842F9883C05886
:102E3000DF4F88508830D0F788EF840F86958695CD
:102E4000869590E8899FE00DF11D1124E058FF4F11
:102E50004770442309F476C0A42FB0E0A65FBD4FAD
:102E60009C910130110541F050F00230110509F03C
:102E700069C08081892706C08081892B03C0909515
:102E80008081892380835EC057FD5CC08E819F81D5
:102E9000481759070CF056C077FF04C0260F371F9C
:102EA00060E070E08C819D81FB01E20FF31F8E17C3
:102EB0009F071CF49C01261B370B121613060CF0FF
:102EC00041C0CA0157FD0796E3E095958795EA95BD
:102ED000E1F79695982F882797958795865E9D4F61
:102EE000860F971F4770552761E070E001C0660F9D
:102EF0004A95EAF7462F0130110541F088F002307B
:102F0000110501F5FC01280F391F15C0FC01280F20
:102F1000391FE217F307B1F08081842B8193F9CF39
:102F20006095FC01280F391FE217F30759F08081E3
:102F300086238193F9CFE217F30721F0808184275C
:102F40008193F9CFDF91CF911F910F9108950F9346
:102F50001F93CF93DF93FC018589823069F0833022
:102F6000E1F0813009F082C0C481D581C41BD50B4A
:102F7000C21BD30BDB0117C084819581DC01A61B2A
:102F8000B70BBD016150710986819781DC01A41BDB
:102F9000B50BAD01421B530B69C0A681B781A61BBF
:102FA000B70B1197EA01B7FD08C186819781A81771
:102FB000B9070CF002C1D7FF04C02C0F3D1FC0E0C1
:102FC000D0E084819581AE01420F531F841795078D
:102FD0001CF49C012C1B3D0B121613060CF0EDC0CB
:102FE000CD01B7FD079643E0959587954A95E1F7A2
:102FF0009695982F882797958795865E9D4F8C0F7D
:103000009D1FA770BB2741E050E00A2E01C0440F6E
:103010000A94EAF7642F0130110549F098F0023064
:10302000110509F0CAC0FC01280F391F17C0FC01A7
:10303000280F391FE217F30709F4BFC08081862BE0
:103040008193F8CF4095FC01280F391FE217F30751
:1030500009F4B3C0808184238193F8CFE217F3078A
:1030600009F4ABC0808186278193F8CF77FDA5C096
:1030700084819581681779070CF09FC057FF04C0C1
:10308000240F351F40E050E086819781FA01E20F5E
:10309000F31F8E179F071CF49C01241B350B12167F
:1030A00013060CF08AC0522F842F8695869586953C
:1030B000FB01B0E88B9FE00DF11D1124E65EFD4F92
:1030C000477069F168E0641B862F90E0EC01CE5EEA
:1030D000DD4F4881261760F4DC01A21BB1098FEF98
:1030E00090E00A2E02C0959587950A94E2F748234E
:1030F0000130110539F048F00230110551F480819A
:10310000842706C08081842B03C04095808184235E
:103110008083561708F451C0561BE058FF4F5830B3
:10312000A0F102301105A9F4DF01852F9C91909543
:103130009C93A058BF4F88508830C0F788EF850F08
:10314000869586958695B0E88B9FE00DF11D11243C
:1031500019C081E00130110509F080E0982F9195A8
:10316000EF01852F9883C058DF4F88508830D0F703
:1031700088EF850F86958695869590E8899FE00D66
:10318000F11D1124E058FF4F57705523B1F0A52FC2
:10319000B0E0A65FBD4F9C910130110539F048F0B9
:1031A0000230110551F48081892706C08081892B66
:1031B00003C09095808189238083DF91CF911F91F7
:1031C0000F910895CF92DF92EF92FF920F931F938A
:1031D000CF93DF937C018B01EA01690177FDA0C0E9
:1031E0000E946716081719070CF09AC0D7FD98C0FF
:1031F000C7010E946B16C817D9070CF091C0C70110
:103200000E946416823009F07FC0F70184819581A5
:103210009C01201B310B8901015011098681978186
:10322000FC01EC1BFD0BEF0121970BC0813049F431
:10323000F701848195818C1B9D0BE8018C01015065
:103240001109F1E0CF16D10431F010F132E0C316CC
:10325000D104E1F165C0FE01D7FD379683E0F59515
:10326000E7958A95E1F7F695FE2FEE27F795E79516
:10327000E00FF11FE65EFD4FC770DD2781E090E0B3
:103280000C2E01C0880F0A94EAF79081982B3AC05F
:10329000FE01D7FD3796A3E0F595E795AA95E1F7EE
:1032A000F695FE2FEE27F795E795E00FF11FE65E06
:1032B000FD4FC770DD2781E090E00C2E01C0880F24
:1032C0000A94EAF78095908198231CC0FE01D7FDEF
:1032D000379663E0F595E7956A95E1F7F695FE2F49
:1032E000EE27F795E795E00FF11FE65EFD4FC770FB
:1032F000DD2781E090E00C2E01C0880F0A94EAF7E8
:103300009081982790830CC0833009F08FCFF7010C
:1033100086819781801B910B8E01EC01219791CFC3
:10332000DF91CF911F910F91FF90EF90DF90CF90A1
:1033300008951F93CF93DF93EC01162F40E250E0E6
:1033400060E870E00E94B91389E394E09983888370
:103350008FEF8C8F88A38E8F8D8F1F8FDF91CF91F2
:103360001F91089580E092E0EAE1F2E0DF019C0124
:103370001D9221503040E1F70895FC0181A188237E
:1033800039F06EBD00000DB407FEFDCF8EB5089577
:1033900088E090E030E8A4A1B5A14C9123A5209548
:1033A00024232C93A2A1B3A122A5432F462321F0CD
:1033B0004C91422B4C9304C04C91209524232C9388
:1033C000A4A1B5A12C9143A5242B2C93369501974C
:1033D00011F708951F93CF93DF93EC01162F8C8D77
:1033E0008F3F09F1EEA1FFA180819CA5892B8083ED
:1033F000E8A5F9A590818DA5809589238083EEA10C
:10340000FFA190818CA5809589238083CE010E94A5
:10341000BD19EEA1FFA180819CA5892B8083DF913E
:10342000CF911F9108958A8D682F772767FD70953A
:1034300088E69DE00E94DD2660E088E69DE00E942F
:103440008A26612F88E69DE00E948A2688E69DE014
:10345000DF91CF911F910C94F2260F931F93CF937E
:10346000DF93EC01162F022F6B8F4A8F8C8D8F3FCD
:1034700009F489C061E08E8D0E94242A61E088A150
:103480000E94242A88A1992787FD9095FC01E8567F
:10349000F84FE491F0E0EE0FFF1FE454F84F259150
:1034A00034913FA32EA3FC01EC58F84F84918CA7D4
:1034B0008E8D992787FD9095FC01E856F84FE49191
:1034C000F0E0EE0FFF1FE454F84F2591349139A737
:1034D00028A7FC01EC58F84F84918DA789A1811190
:1034E00034C061E08C8D0E94242A61E08D8D0E94A1
:1034F000242A8D8D992787FD9095FC01E856F84F79
:10350000E491F0E0EE0FFF1FE454F84F2591349161
:103510003DA32CA3FC01EC58F84F84918BA78C8D14
:10352000992787FD9095FC01E856F84FE491F0E06B
:10353000EE0FFF1FE454F84F259134913BA32AA3CB
:10354000FC01EC58F84F84918AA789A18823F9F0EF
:103550000E941C268091670D882381F0813051F4F0
:103560008DB38093650D9DB38091660D8095892301
:103570008DBB04C08FB78093650DF89480E58CBD3A
:1035800081E08DBD04C088E69DE00E94C92600232D
:10359000F1F08F8D87FD1BC061E00E94242A61E05D
:1035A0008F8D0E945D2A61E070E080E090E00E94D3
:1035B0003C2960E08F8D0E945D2A6AE070E080E027
:1035C00090E00E943C2961E08F8D0E945D2A6EEAA6
:1035D000CE010E94EA1965EDCE010E94EA1960E869
:1035E000CE010E94EA1968EACE010E94EA196FE151
:1035F000CE010E94EA1963EDCE010E94EA1960E053
:10360000CE010E94EA1960E4CE010E94EA196DE839
:10361000CE010E94EA19113011F460E101C064E1A9
:10362000CE010E94EA1960E2CE010E94EA1960E030
:10363000CE010E94EA1961EACE010E94EA1968EC03
:10364000CE010E94EA196AEDCE010E94EA1962E0F9
:10365000CE010E94EA1961E8CE010E94EA196FE8E2
:10366000CE010E94EA1969EDCE010E94EA191130DB
:1036700011F462E201C061EFCE010E94EA196BED24
:10368000CE010E94EA1960E4CE010E94EA1964EAC0
:10369000CE010E94EA1966EACE010E94EA196EE2A2
:1036A000CE010E94EA196FEACE01DF91CF911F91FE
:1036B0000F910C94EA19662311F067EA01C066EADB
:1036C0000C94EA19DF92EF92FF920F931F93CF931E
:1036D000DF93EC0161E20E94EA1960E0CE010E94F2
:1036E000EA196FE7CE010E94EA1962E2CE010E9458
:1036F000EA1960E0CE010E94EA1963E0CE010E945F
:10370000EA198C8D8F3F31F1EEA1FFA180819CA53C
:10371000892B8083E8A5F9A580819DA5892B8083CD
:10372000EEA1FFA190818CA58095892380830AE179
:1037300012E0F80161918F01CE010E94BD19F4E001
:103740000A311F07B1F7EEA1FFA180819CA5892B4B
:10375000808337C0D090B8008CE08093B8000AE135
:1037600012E06A8D772767FD709588E69DE00E94DC
:10377000DD26E091680DF091690D0190F081E02D5A
:1037800060E488E69DE01995E12CF12CF801EE0D3E
:10379000FF1D608188E69DE00E948A268FEFE81A6F
:1037A000F80AE0E1EE16F10489F788E69DE00E9450
:1037B000F226005F1F4FF4E00A311F0791F6D09206
:1037C000B800DF91CF911F910F91FF90EF90DF90A4
:1037D0000895CF92DF92EF92FF920F931F93CF93B2
:1037E000DF93CDB7DEB72C970FB6F894DEBF0FBED0
:1037F000CDBF8C01DC011F968C918230A1F038F492
:10380000882371F08130D9F482E090E014C08032D6
:1038100069F0813271F0813191F485E090E00BC064
:1038200081E090E008C083E090E005C086E090E091
:1038300002C087E090E09093540B8093530B10925A
:10384000BE0B1092BD0B4AE0F8016089CE010796CD
:103850000E942C2F6DE474E0CE0101960E94832E0D
:10386000BE01695F7F4FCE0101960E94F82FBC0117
:1038700081E39EE00E94682DCE0101960E94152EE4
:10388000CE0107960E94152ED8011C96CC908091EF
:10389000530B9091540B019701F567E574E081E3B8
:1038A0009EE00E944B2DE12CF12CD12CEC14FD0458
:1038B00084F4D8011A96ED91FC911B97EE0DFF1D33
:1038C000608181E39EE00E944D2DBFEFEB1AFB0A61
:1038D000EDCF81E39EE00E94542D2C960FB6F89414
:1038E000DEBF0FBECDBFDF91CF911F910F91FF9033
:1038F000EF90DF90CF900895AF92BF92CF92DF927A
:10390000EF92FF920F931F93CF93DF9300D000D0DD
:10391000CDB7DEB77C01FC01C480D5806BEB74E0D1
:1039200081EC9BE00E94FB2E6BEB74E087EC9BE04C
:103930000E94FB2E6BEB74E08DEC9BE00E94FB2E53
:103940006BEB74E083ED9BE00E94FB2E00E010E047
:10395000B801C7010E9455308A3319F00C151D05B6
:103960002CF1B801C7010E94553098012F5F3F4FDD
:1039700059018A3309F448C00C151D050CF044C0E8
:10398000B801C7010E945530682FCE0101960E94F0
:10399000132FBE016F5F7F4F87EC9BE00E94DD2FEE
:1039A000CE0101960E94152E8501DBCFB801C7011B
:1039B0000E945530682FCE0101960E94132FBE0140
:1039C0006F5F7F4F81EC9BE00E94DD2FCE0101965F
:1039D0000E94152E0F5F1F4FBBCF0C151D05F4F471
:1039E000B801C7010E945530682FCE0101960E9490
:1039F000132FBE016F5F7F4F8DEC9BE00E94DD2F88
:103A0000CE0101960E94152E8501B801C7010E94C2
:103A10005530F80131965F018A33F9F68501B80116
:103A2000C7010E9455308D32D1F00C151D05BCF434
:103A3000B801C7010E945530682FCE0101960E943F
:103A4000132FBE016F5F7F4F83ED9BE00E94DD2F40
:103A5000CE0101960E94152E0F5F1F4FE0CF67EC3D
:103A60007BE081E39EE00E94682D26960FB6F894D5
:103A7000DEBF0FBECDBFDF91CF911F910F91FF90A1
:103A8000EF90DF90CF90BF90AF900895EF92FF92AC
:103A90000F931F93CF93DF93CDB7DEB7CA57D109EA
:103AA0000FB6F894DEBF0FBECDBF8C018091BF0B67
:103AB0009091C00B892BF1F18AE00E94530AD80142
:103AC00019962C9130E040E250E060E070E04983CC
:103AD0005A836B837C83FE0135968AE3DF011D9256
:103AE0008A95E9F7BE016F5F7F4F80E090E0821713
:103AF00093076CF4D8011796ED91FC911897E80F95
:103B0000F91F4081FB014193BF010196F0CFBE0137
:103B10006F5F7F4FCE0181599F4F0E94832EBE0160
:103B200061597F4F81E39EE00E94682DCE0181594B
:103B30009F4F41C0D8011996EC90F12C6BEB74E0CB
:103B4000CE018B589F4F0E94832EAE014F5F5F4F77
:103B500080E090E08E159F056CF4D8011796ED91EA
:103B6000FC911897E80FF91F2081FA012193AF010A
:103B70000196F0CF8AE00E94530ABE016F5F7F4F2B
:103B8000CE0181599F4F0E94832ECE0181599F4FB4
:103B90000E947C1CCE0181599F4F0E94152ECE01A0
:103BA0008B599F4FFE0131961192E817F907E1F703
:103BB000CE018B589F4F0E94152E81E0C658DF4FD3
:103BC0000FB6F894DEBF0FBECDBFDF91CF911F912E
:103BD0000F91FF90EF900895EF92FF920F931F9334
:103BE000CF93DF93EC01198218821B821A821D8207
:103BF0001C821E821F82188619866BEB74E00A965F
:103C00000E94832E6BEB74E0CE0140960E94832EBF
:103C10001F8A1E8A1B8E1A8E1D8E1C8E8E01025EBE
:103C20001F4F78018CE3E80EF11C6BEB74E0C801C8
:103C30000E94832E0A5F1F4F0E151F05B1F76BEB15
:103C400074E0CE018A579F4F0E94832E6BEB74E085
:103C5000CE0184579F4F0E94832E6BEB74E0CE0100
:103C60008E569F4F0E94832E6BEB74E0CE018856D8
:103C70009F4F0E94832EFE01E256FF4F1082118259
:103C800012821382349610823196118210823296FB
:103C900081E090E0918380833296108211821282BB
:103CA000138234961082118212821382349648EE67
:103CB00053E060E070E040835183628373836BEB79
:103CC00074E0CE018D549F4F0E94832EFE01E75475
:103CD000FF4F118210826BEB74E0CE0185549F4F31
:103CE0000E94832EFE01EF53FF4F10821182128239
:103CF00013828EB3CA53DF4F8883DF91CF911F9118
:103D00000F91FF90EF900895EF92FF920F931F9302
:103D1000CF93DF93EC0185549F4F0E94152ECE0167
:103D20008D549F4F0E94152ECE0188569F4F0E94A2
:103D3000152ECE018E569F4F0E94152ECE01845710
:103D40009F4F0E94152ECE018A579F4F0E94152E1D
:103D50007E018EE1E80EF11CE114F10461F08E01A8
:103D6000065A1F4F0E151F0531F006501109C801E4
:103D70000E94152EF7CFCE0140960E94152ECE013F
:103D80000A96DF91CF911F910F91FF90EF900C94C5
:103D9000152E8AE29BE00E94152E82E39BE00E9492
:103DA000152E8BE39BE00C94841E2F923F924F9232
:103DB0005F926F927F928F929F92AF92BF92CF92BB
:103DC000DF92EF92FF920F931F93CF93DF93CDB7C4
:103DD000DEB729970FB6F894DEBF0FBECDBF8C01BA
:103DE0007B012DB63EB6FC01EC57FF4F80819181DF
:103DF00098012E573F4F5901F901019709F0BFC0B3
:103E000080819181892B09F029C16BEB74E0C70196
:103E10000E94253081113EC06DB67EB6B701CE013D
:103E200001960E94E62ECD80DE80CE0101960E9492
:103E3000152E2DB73EB72C193D090FB6F8943EBF8D
:103E40000FBE2DBF8DB79EB701964C01412C512C52
:103E50004C145D045CF4B201C7010E945530F401BA
:103E600081934F01FFEF4F1A5F0AF2CFB7018AE249
:103E70009BE00E94CF2EB80165547F4FC801409649
